:100000005FC040C278C077C076C075C074C073C08E
:1000100072C071C070C06FC06EC06DC06CC06BC06C
:100020006AC069C068C067C066C065C064C063C09C
:1000300062C061C0040309042203770077007700DF
:100040002E00720065006300750072007300690085
:100050006F006E002E006A00700010035500530000
:1000600042002D0032003300320012011001020064
:100070000008C016E1050001010200010902430069
:10008000020100803209040000010202010005247F
:1000900000100104240202052406000105240103C6
:1000A00001070583030800FF09040100020A00009C
:1000B0000007050102080000070581020800000092
:1000C00011241FBECFEFD2E0DEBFCDBF11E0A0E014
:1000D000B1E0ECEFFAE002C005900D92AC30B10750
:1000E000D9F712E0ACE0B1E001C01D92AC3DB10720
:1000F000E1F730D401C584CFE9E6F0E08081836088
:100100008083E89A8BE48093220180934D018AE5F5
:100110008093210180934C0108951F93DC01162FD9
:1001200080914C0184FF17C080914D0198E8892788
:1001300080934D01912FEEE4F1E08D9181939150E8
:100140001916DCF3612F8EE491E098D11C5F1093B7
:100150004C011F9108958AE580934C01EBCF1F93CA
:10016000DC01162F8091210184FF17C080912201AC
:1001700098E8892780932201912FE3E2F1E08D91A5
:10018000819391501916DCF3612F83E291E076D1CF
:100190001C5F109321011F9108958AE5809321012E
:1001A000EBCF1F93CF93DF9360913201635067FDD4
:1001B0001AC080912F01CCE0D0E0C81BD109CA5CE5
:1001C000DE4F80912E01803108F481C08D3209F418
:1001D00081C080910C0187FDADC08091320118165D
:1001E00014F4109232018091000184FF4AC06091A2
:1001F00001016F3F09F445C0693070F168506093A8
:1002000001018091160198E889278093160168E022
:1002100080910C0187FD9EC0209130013091310109
:1002200086FF7FC0A7E1B1E080E090E0F901E80F30
:10023000F91FE491ED9301966817C1F76150862F7D
:1002400090E06F5F0196820F931F9093310180932E
:100250003001162F1C5F0BC0109201018091160116
:1002600098E8892780931601662391F614E087E1C8
:1002700091E004D11C3019F08FEF809301011093AD
:10028000000189B18C70F9F489B18C70E1F489B105
:100290008C70C9F489B18C70B1F489B18C7099F407
:1002A00089B18C7081F489B18C7069F489B18C70DA
:1002B00051F489B18C7039F489B18C7021F41092A9
:1002C000330110922D01DF91CF911F910895CE013E
:1002D0001CD383CF683009F080CF83EC8093160164
:1002E0008AE58093000110920C018881807609F0E4
:1002F00053C09A8110921F0189818823B9F5109209
:10030000200122E08FE191E0909331018093300150
:100310008F818823E9F49E819217D0F49093010194
:100320005CCF962FD901E7E1F1E08D918193915057
:10033000E1F784CFCE0196D38F3F31F0882309F4C3
:100340004CCF1092010149CF8EE18093000145CF3F
:10035000922FE4CF87E191E0C0D2682F893008F472
:1003600061C08FEF809301011EE189CF853011F1CB
:10037000863041F18830E1F1893009F441C08A309A
:10038000D9F18B3029F48BE48093220180934D01C5
:1003900020E08FE191E0B8CFCE017FD2282F2F3F10
:1003A00009F0B6CF888187FD0BC09FEF80E880936E
:1003B0000C01B4CF9093330120E08FE191E0A4CF02
:1003C0009E81F4CF8B81813029F18230F9F0833026
:1003D00029F020E080E480930C01E1CF992329F5F6
:1003E00084E390E0909331018093300124E0F2CFD8
:1003F00021E085E391E088CF21E08FE191E084CF97
:100400009093350120E08FE191E07ECFCE0130D294
:10041000282FE0CF8AE690E090933101809330015D
:1004200022E1D8CF182F1C5F22CF913051F09230AB
:1004300081F68AE590E0909331018093300120E1CC
:10044000C9CF88E390E0909331018093300122E29C
:10045000C1CFA82FB92F80E090E041E050EA60952D
:100460006F5F58F42D9138EF82279795879510F09C
:10047000842795273F5FC8F3F3CF0895EADF8D9374
:100480009D930895CF93CFB7CF934B9BFECF4B9BBC
:1004900009C04B9B07C04B9B05C04B9B03C04B9BAC
:1004A00001C0A6C0DF93C0912F01DD27CA5CDE4FDB
:1004B0004B9B02C0DF91EBCF2F930F931F9309B19A
:1004C0002FEF03FB20F94F933F9319B14FEF012713
:1004D00003FB21F93BE031C04E7F012F19B12160B0
:1004E00028C0102F4D7F2260000009B129C04B7F2A
:1004F0002460012F000019B12BC019B1477F28607B
:100500002AC04F7E09B120612CC04F7D19B12062F5
:100510002FC04F7B09B1206432C0422709B14993F3
:100520004FEF0000102713FB20F919B11C70C9F11F
:10053000297F91F2012703FB21F909B1237F89F279
:10054000315058F1102713FB22F919B1277E79F2A7
:10055000012703FB23F92F7C81F209B1102713FB3C
:1005600024F92F7971F200C019B1012703FB25F995
:100570002F7359F200C009B1102713FB26F922305E
:1005800040F200C019B1012703FB27F9243028F6F7
:100590004F77206819B10000F9CF11E01CBB00278C
:1005A0001CC03B503195C31BD04011E01CBB0881DF
:1005B000033C11F10B3401F120912D011981110F30
:1005C0001213EDCF4A81441F093659F10D3211F053
:1005D000013E29F74F7009F0042F009334013F9139
:1005E0004F911F910F912F91DF91CCB3C0FD4DCF53
:1005F000CF91CFBFCF91189500913401002379F3AB
:10060000109132011123F9F53430FAF130933201AF
:1006100000932E0110912F013BE0311B30932F01ED
:1006200034C000913201013074F50AE54F7049F48D
:100630003091000134FD2BC000930001C6E1D1E0F0
:100640002AC0433049F03091210134FD20C000938D
:100650002101C2E2D1E01FC030914C0134FD17C02E
:1006600000934C01CDE4D1E016C0052710E00BB992
:100670001FC0052722C0052727C005272CC0052736
:1006800010E00BB933C04AE503C042ED01C0432F6F
:10069000C4E1D0E032E01AB11C605B9A0BB11AB928
:1006A0005F935CE020E820FF05270BB9279517959D
:1006B0001C3FD8F620FF052727950BB917951C3F3F
:1006C000C0F620FF0527279517950BB91C3F98F614
:1006D00020FF0527279517951C3F0BB970F600C022
:1006E000499120FF05270BB9279517951C3F38F630
:1006F00020FF052727950BB917951C3F38F520FFDC
:100700000527279517950BB91C3F10F520FF0527E6
:10071000279517951C3F0BB9E8F4242F3A9519F645
:10072000037F5F910BB910913301110FC651D04077
:1007300011F010932D0111E01CBB08601AB1137F5A
:10074000402F437F0BB91AB94BB949CF0527D3CFF7
:100750000527D8CF0527DDCFBF92CF92DF92EF924A
:10076000FF920F931F936B017C01B42E122FCC0CC0
:10077000DD1CEE1CFF1CCC0CDD1CEE1CFF1CCC0C8D
:10078000DD1CEE1CFF1C60E07BE187EB90E0A70125
:10079000960190D121503040404050408091C0009F
:1007A00082608093C0001092C10081E0B816F9F019
:1007B0004B2D4295407F802F90E00597880F991F21
:1007C0001695110F110F110F182B412B4093C200DA
:1007D0002093C4003093C50088E18093C1001F912D
:1007E0000F91FF90EF90DF90CF90BF90089540E37E
:1007F000E2CF8091C00085FF16C02091DA0290916F
:10080000DB02291781F0E92FF0E0E75AFD4F8081E4
:100810008093C600E92FEF5FEF77E093DB028091D2
:10082000320187FD19C08091C00087FF0895809133
:10083000C0002091C6008C71C9F7E09158029E2F2C
:100840009F5F8091D902981789F3F0E0E85AFE4F34
:10085000208390935802089520952E0F2F772930EA
:1008600010F310923201DFCF8091C000807808959C
:10087000FC018381813041F08CE790E0909331015D
:100880008093300183E408958AE690E090933101EB
:100890008093300180916A000895FC012081822FAD
:1008A0008076803211F080E008959181892F805206
:1008B000823048F0923249F027FDF5CF81E08093F5
:1008C0000D0180E008958FEF089580910E01882337
:1008D00099F782E080930E01EFCFFC018091120125
:1008E00080838091130181838091140182838091A0
:1008F0001501838380910F0184838091100185838A
:1009000080911101868387E00895DC016623E9F078
:100910009091DB02E091DA022D91EF5F8E2F8F77BD
:10092000E150891739F0F0E0E75AFD4F20838093BA
:10093000DA02E82F615081F791509E1B9F77993022
:1009400018F48FEF8093320108959091DB02E091CB
:10095000DA02F2CF0F931F932EE088E190E00FB6FA
:10096000F894A895809360000FBE2093600083EFF9
:100970008BB98CE08AB924E148EC5FEAA895CA01FA
:100980000197F1F72150D1F71AB880EC92E1A0E07D
:10099000B0E08093120190931301A0931401B093DF
:1009A000150110920F011092100188E0809311013F
:1009B00008E040E060EC72E180E090E0CDDE109273
:1009C000DB02109258021092D9021092DA0294DBE4
:1009D00010920E0110920D01789411E018C0062FAC
:1009E000091B29F580910D01882369F010920D01F2
:1009F000892F90E0602F885A9E4FB1DB8091D902F9
:100A0000800F8093D90290910E019923B1F4A8959B
:100A1000C8DBEFDE8091210184FFF5CF9091D902F0
:100A2000609158026917D8F6092F0195D9F208305C
:100A3000E8F210930D0108E0DBCF80914C0184FFB8
:100A4000E6CF923051F062E08AE091E066DB80917F
:100A50000E01815080930E01DACF68E082E091E0D0
:100A60005CDBF5CF0F93FC018081809312018181C3
:100A700080931301828180931401838180931501F7
:100A800060911201709113018091140190911501F0
:100A90000091110120910F01409110015DDE109233
:100AA000DB02109258021092D9021092DA0281E011
:100AB0000F910895A1E21A2EAA1BBB1BFD010DC0C8
:100AC000AA1FBB1FEE1FFF1FA217B307E407F507FE
:100AD00020F0A21BB30BE40BF50B661F771F881FDA
:100AE000991F1A9469F760957095809590959B0170
:0C0AF000AC01BD01CF010895F894FFCFC8
:0C0AFC005AFFA1200000000002000300CF
:00000001FF
